:030000000219FDE5
:03000B000200AA46
:03002B0002015F70
:03005B000202F9A5
:030073000202E6A0
:1000800002030406080C10182030406080040608A3
:100090000C10182030406080A0C00003070F1F0D17
:1000A0000D04050D050305030302C2AFC0D0C0E077
:1000B000206214E5256009E473E525F4F58AD2622F
:1000C000D0E0D0D0D2AF3285268AC262E526F46075
:1000D0003030682620720DD0E0D0D0C295C294C2D4
:1000E00093D2AF32C295C294C293206F0D20650A9D
:1000F000740AD5E0FDE57BF45290D0E0D0D0D2AFC9
:1001000032758A00C28DD26201FA01B930680520C9
:100110006502D29501B9306805206502D29401B913
:10012000306805206502D29301B9D29230680A2066
:1001300065077408D5E0FDD29501B9D29130680AFF
:100140002065077408D5E0FDD29401B9D290D2920F
:1001500030680A2065077408D5E0FDD29301B9C262
:10016000AFC2AD53E6EFC0D0C0E0D2D3D2AFC2CE63
:10017000E52A600720744F152A21C67800790020EF
:10018000742EE580307E01F430E70278FF53DACF39
:10019000207E0343DA20307E0343DA10C2D8C271D6
:1001A000E580307E01F430E70279FFC3E89970CB37
:1001B000306103752A18207403752A18885CD27080
:1001C000E86003755F0020740DE52B6004152B219A
:1001D000D643DA01C2D82070024145A85C206102F2
:1001E000C2702074367982B70431C3E894F04003BA
:1001F00074F0F8E8C4540F28F87984B70302411B5F
:10020000C313C3138721200802C313200A06C3C8DF
:1002100098F8411B28F8500374FFF88822E52D5404
:10022000066022206B1FE536C333C333F8E564C391
:1002300013C313F9C3952240028922E82522F5222F
:1002400050037522FF7882B60459852224A824C35E
:10025000E52495614002A861C3E895634002A86364
:100260008825E56670024196C3E8AA669A5003E8BD
:10027000FAE4F9EAC333FBE568F45B29400D25672E
:10028000F8E56760021567400B41960AC3E5679A77
:100290005002056778FF8826C26FC3E52694F840B0
:1002A00002D26F20CF0AD0E0D0D043E610D2AD32D8
:1002B000C2CF053A7801E52A6005307402152AC3D9
:1002C000E55C94014005755F0041DC75600075696F
:1002D00000E55F2401F55F5003755FFFD0E0D0D0EB
:1002E00043E610D2AD32C2AF53E67F7592FA7593F2
:1002F000FFC260759104D2AF32C2AF53E6EFC2AD18
:10030000C0D0C0E0C0F0D2D3D2AFA8FBA9FCC2D805
:10031000307102616053DACF207E0343DA10307E01
:100320000343DA20D271E580307E01F420E70261D8
:100330003788278928A18D53DACF207E0343DA201E
:10034000307E0343DA10C2D8C271307402A17978CA
:1003500000E580307E01F430E702A179885CA1617C
:1003600053DACF207E0343DA20307E0343DA10C213
:1003700071206102813953DACF207E0343DA1030D5
:100380007E0343DA20C2D8D27188578958C3E895D2
:1003900055F8E99556F97B007E087A00C3E8948CFD
:1003A000E994005005755B00812B882178A2E6A8AE
:1003B000216055C3E894C8E994005008E4D2E4FBF6
:1003C0007A0A8106C3E89468E994015008E4D2E30C
:1003D000FB7A0F8106C3E894D0E994025008E4D276
:1003E000E2FB7A1E8106C3E894A0E994055008E474
:1003F000D2E1FB7A3C8106C3E89498E9940850085E
:10040000E4D2E0FB7A787E00C3E89559FCE9955A7E
:10041000FD30E70AECF42401FCEDF43400FD755BDB
:1004200000C3EC9AED9E5003755B018859895A858B
:1004300057558558567802A161C3E89527F8E99584
:1004400028F9307C02A145307B02A145307A02A117
:100450003E207502815CE9FDE8FC817BE9C313F96C
:10046000E813F8307902A13EE9C313F9E813F83034
:0F0470007802A13EE9C313FDE813FC20612CC301
:10047F00EC941CED940240028192ED701EC3EC943B
:10048F00C850180529E52970021529C3E529940AD2
:10049F005002A179755C00D270A179E5296002152F
:1004AF00297888E6F97400207F087896B9030278D6
:1004BF009EE624FAFEE43400FFC3EC9EFCED9FFDA4
:1004CF009208B90310A2085007207609D27681E46A
:1004DF00307602C276A2085016B9030DECF424014F
:1004EF00FCEDF43400FD0204FE78007900A145B95B
:1004FF000315EC33FCED33FDC3EC940AFCED9400D3
:10050F00FD50047C007D00C3EC94FFED9400400689
:10051F0078FF7900A145EC8572F0A4C5F0A2F733FE
:10052F00F87900400302056178FF7900020561E95F
:10053F00C313F9E813F8307C0EE9600278FFC3E8C3
:10054F001338F8E43400F9C3E894FFE9940040024B
:10055F0078FF885CD270206102A179741FF4552F47
:10056F004BF52FC274EB7002D274752A18307403D6
:10057F00752A0A306102A18D20740353DAFE2074AC
:10058F0003752B06D0F0D0E0D0D0D2AD43E61032B9
:10059F0079010205BD79030205BD790A0205BD790E
:1005AF001E0205BD79640205BD79C80205BD781725
:1005BF00E4D5E0FDD8FAD9F6227A147B780205E467
:1005CF007A107B8C0205E47A0D7BB40205E47A0B7A
:1005DF007BC80205E4E573D5E001227902E4D291EC
:1005EF00D5E0FDD294D5E0FDC294D5E0FDC291D502
:1005FF00E0FDE920E002D29530E002D293E573D519
:10060F00E0FDE920E002C29530E002C2937496D576
:10061F00E0FDD9C9EAF8D5E0FDD8FBDBB8D29122CD
:10062F00C37C007D0075F00005F0EA33FAEB33FB75
:10063F0050F6EB13FBEA13FAC3E9FFE8FEE89AF86A
:10064F00E99BF95004EFF9EEF8B3EC33FCED33FD11
:10065F00D5F0DFEDF9ECF822E889F08A20D2D4F852
:10066F00A9F07B0030F70B7BFFF42401F8E9F43499
:10067F0000F9E88520F0A4ADF0F8E98520F0A4AFEB
:10068F00F0FEED2EF974003FFA7C04C3EA13FAE989
:10069F0013F9E813F8DCF48BF030F70AE8F42401CF
:1006AF00F8E9F43400F9E889F0C2D4F8A9F0227817
:1006BF0082B60403020719C3E55C940140030206E6
:1006CF00E3852224E4F544F545F546F547F548C2A0
:1006DF006E0207197882E6FCD26EE522F523783890
:1006EF0079C7AA40AB41C3EB13FBEA13FAEC1460D2
:1006FF0013C3EB13FBEA13FAEC14146007C3EB13E9
:10070F00FBEA13FAD12F8844894522C3E544952388
:10071F00F8E5459400F9500CC3E89480E994FF4044
:10072F001602074AC3E8947FE99400500302074A70
:10073F00787F790002074A788079FF8849894A22B1
:10074F00E5492546F8E54A3547F9854A20E430075B
:10075F0001F43548FA30E709C3EA94F0401502076F
:10076F0088C3EA940F500302078878FF79FF7A0F46
:10077F00020788780079007AF0C3E5249561500A62
:10078F00C374019524500B0207A6E54A20E70E0219
:10079F0007A6E54A30E706884689478A482278A5A2
:1007AF00E6FAC3E54933F8E54A33F9D167E930E7AB
:1007BF000BC3E89480E994FF4013E1E0C3E8947F12
:1007CF00E994005002E1E0787F7900E1E0788079E8
:1007DF00FFE820E715C3E52398F84009C3E8940123
:1007EF0040030208077801020807E8F424012523D3
:1007FF00F8400302080778FF884B2278A6E6FAA88C
:10080F0047A948120667E930E70CC3E89401E99459
:10081F00FF401602083CC3E894FFE994005003021E
:10082F00083C78FF790002083C780179FFE920E75E
:10083F0015C3E54B98F84009C3E89401400302083B
:10084F00637801020863E8F42401254BF8400302A2
:10085F00086378FF88242278FF20692879A1E76050
:0E086F0023E541601F74FF8541F0848539F058
:10087D00306A0375F005A4F8C5F0600278FFC3E88F
:10088D0095645002A864886322C3E5409440E54115
:10089D009401E56350031401A7046002F56322027D
:1008AD0008AF2275E890227883E6FF30EDF9A8BDF8
:1008BD00A9BE0570C3E57094084052757000E9FA41
:1008CD0079A0E76044EA7007E571601B0208E8C390
:1008DD00E895716010E5715006600C140208F4047F
:1008ED0060F90208F4E571F571C3946D401B7561F3
:1008FD00C0C394044013756180C39404400B7561AB
:10090D0040C39404400375610075BB0622E5612464
:10091D0010500274FFF5617982B704022141C3A81A
:10092D0061E524985002A824C3E895634002A863AA
:10093D0088258826E570B4070375BB1022743279BB
:10094D00A787F0A4C5F0A2F733F8C3E8956140027C
:10095D00A86188228824882588268864227540000D
:10096D007541F022C2AF75C820A8CCA9CDAA3A30E6
:10097D00CF010A75C824D2AFAB3BAC3C883B893C58
:10098D00C3E89BF8E99C206908F930660241822191
:10099D00DCAD3D8A3DF9EA9DFA600678FF79FF21CD
:1009AD00C1AE3EAF3F8B3E8C3FA83BA93CC3E89EFA
:1009BD00F8E99FF9C3E54113FBE54013FAE82AF581
:1009CD0040E93BF54150067540FF7541FF4129AAAD
:1009DD0040AB41AC40AD417E047F02C3EB9404407B
:1009ED000D1E1FC3EB94084005206A021E1FC3EDA8
:1009FD0013FDEC13FCDEF7C3EA9CFAEB9DFBEF60F5
:100A0D0009C3E913F9E813F8DFF7EA28FAEB39FB24
:100A1D008A408B4150067BFF8B408B41C3EB940288
:100A2D005002D2663069047F0341547892E6FFC3C9
:100A3D00E537948240110FC3E53794A040010FC3F1
:100A4D00EF940640027F057E02E541C4540FF9E59F
:100A5D0041C454F0F8E540C4540F28F8C3E89EFA99
:100A6D00E99400FB4009C3EA9402EB940050047A28
:100A7D0002E4FB41CEAA40AB41EBC4FEEAC4540FE5
:100A8D004EFCC3EA9CFAEB9400FBC3E813C313F8C6
:100A9D00EA28FAEB3400FB8A408B41C3EB94024009
:100AAD0002C2667802EBC4FE7B00EAC4540F4EFA14
:100ABD00C3EA98FA4005C3940250027A027892E68E
:100ACD00FF30600241CE855192855293D26043E64C
:100ADD0080C3E49AF8E49BF9306602615AE8FAE9BA
:100AED00FBD3E913FDE813FC88518952C3EF94033E
:100AFD006038EF20E00DE82CF8E93DF9ECFAEDFB5C
:100B0D00020B23E828F8E939F9C3E82402F8E9349F
:100B1D0000F97AFE7BFFC3EF9403400E8A538B548A
:100B2D00884D894E8C4F8D50618E885389548A4DD6
:100B3D008B4E8C4F8D503069127553F07554FF7577
:100B4D004FF07550FF7551F07552FF618EE8FAD375
:100B5D00E813FC8851C3EF94036020EF20E007E811
:100B6D002CF8ECFA617AE8282402F87AFEC3EF94A7
:100B7D000340088A53884D8C4F618E88538A4D8C63
:100B8D004FE568C3335002646BF5683060026198BD
:100B9D00753402D26043E680E52D54066034A840DA
:100BAD00A941C3E913F9E813F8C3E913F9E813F8F8
:100BBD00306904E92440F9C2AF53E67F759100C353
:100BCD00E498F594E499F595759104D26043E68027
:100BDD00D2AF22D264754300752000306C037520AE
:100BED0040020BFFD264754300752040306C0375D5
:100BFD00200078017901206620E52D54066002C29F
:100C0D00647914E541C313700104F8C394144002D0
:100C1D007814306904781B791B206010E543600C53
:100C2D00306903D53404D26D81A971A00543E59BCC
:100C3D005440B52002819330690908C3E8994001F9
:100C4D0018812620640A08C3E899400261FF8126B5
:100C5D00C264C2AF53E67F75910030661275940081
:0F0C6D007595F8759104D26043E680D2AF61FFB0
:100C7C00E5417EFFC3334005C3334001FEC3E49E10
:100C8C00759400F5958170C3E5339401500261FFB2
:100C9C0030640261FFD80281A78126C26DC2AF53B6
:100CAC00E67F759100855394855495759104854D17
:100CBC0092854E93D26043E680D2AFE52D54066008
:100CCC0008206A020533020CE5306D0D206C0A20F9
:100CDC006407158115810215A5227800306402780D
:100CEC0001E53775F007A4F9E5F028F5F0E9A2F075
:100CFC0013A2F113A2F213F537C39478500375378E
:100D0C0078C3E53795384008D265C295C294C29332
:100D1C00306002A11C854F92855093D26043E680CF
:100D2C0022207D16C2AF754202D291C2923062026D
:100D3C00D293D2AF759F11020F25C2AF754202D26A
:100D4C0091C290306202D295D2AF759F11020F25DD
:100D5C00307245207D22C2AF75420390013B757BFA
:100D6C0002C293D290D292306204D294A17CC291EE
:100D7C00D2AF759F01020F25C2AF75420390013BA4
:100D8C00757B02C295D292306204D294A19CC2911E
:100D9C00D2AF759F21020F25207D17C2AF7542037C
:100DAC00900116C293306202D294D2AF759F0102A9
:100DBC000F25C2AF754203900116C295306202D264
:100DCC0094D2AF759F21020F25207D16C2AF7542BC
:100DDC0004D292C290306202D294D2AF759F21029B
:100DEC000F25C2AF754204D290D292C292306202E9
:100DFC00D294D2AF759F01020F25307243207D2013
:100E0C00C2AF75420590012A757B04C294D2913011
:100E1C006204D295C124C292D2AF759F11020F25E4
:100E2C00C2AF75420590014C757B01C294D29130D2
:100E3C006204D293C144C290D2AF759F11020F25A8
:100E4C00207D17C2AF75420590010CC2943062022E
:100E5C00D295D2AF759F11020F25C2AF7542059086
:100E6C000120C2943062EBD293D2AF759F11020F66
:100E7C0025207D18C2AF754206D290D292C2913015
:100E8C006202D295D2AF759F01020F25C2AF754297
:100E9C0006D292C291306202D293D2AF759F2102D8
:100EAC000F25307246207D20C2AF75420190014C57
:100EBC00757B01C295D292306204D293C1CCC290A0
:100ECC00D2AF759F21020F25C2AF75420190012A46
:100EDC00757B04C293D290D292306205D295020EE9
:100EEC00EFC292D2AF759F01020F25207D17C2AFC2
:100EFC00754201900120C295306202D293D2AF7537
:100F0C009F21020F25C2AF75420190010CC2933094
:100F1C006202D295D2AF759F01C2652290010A750B
:100F2C007B00C295C294C293D292D291D290C262EB
:100F3C0022788076090876090876040876FF087608
:100F4C00030876FF08760A0876030876010876010E
:100F5C00788C76010876FF0876FF0876FF0876FF16
:100F6C000876FF0876030876FF0876FF0876FF08F8
:100F7C0076250876D0087628087650087604087608
:100F8C00FF08760208760008767A0876FF08760164
:100F9C00087601087600087603087600227887E642
:100FAC00FFC272BF0302D2727888E6C39403600852
:100FBC00C27DE630E102D27DC27E7889E630E10264
:100FCC00D27EC3EF94026008758E01D273020FE1DA
:100FDC00758E00C273227880E6149000809378A5F9
:100FEC00F67881E6149000809378A6F67886E6145D
:100FFC0090008D9378A7F67886E6F539C394025065
:10100C0003753902789CE67538FFB402037538A075
:10101C00B4030375388278A3E61490009A93F566AE
:10102C00120F2822227896E6FA7897E6FB7888E663
:10103C00B40305C3EB940EFB307F047A007BFFC333
:10104C00EB9AFCC3948250027C827572000572ECA0
:10105C008572F0A4C3E5F0947D40F222D27F113169
:0F106C001205AE1205AE7A007B007C101205A4AF
:10107B00E55C2AFA74003BFBDCF37C04C3EB13FB4B
:10108B00EA13FADCF7FEC27F113122757C00757D05
:10109B0000E5EF20E6037520000520903FFFE520DB
:1010AB00146006901DFF1460009304600375EF1627
:1010BB0053D9BF7581C043FF8012059F75EF06435F
:1010CB00B203E5B3240220E70DF521E5E320E006AA
:1010DB008521B343E301120F287580FF75A40075BA
:1010EB00F19075D47F75908775A5BF75F2BF75D5D7
:1010FB000075A60175E241120F28E4F8F6D8FD75CC
:10110B006801120F3D1215F678988673753001C27F
:10111B00AF1205B81205C81205AE1205CF1205AEF7
:10112B001205D61205AEC2AF757C00757D0078FA3C
:10113B0079FA308707D9FBD8F7021C00120FA912D6
:10114B000FE21130113178988673120F28758810C1
:10115B0075890275C82475910475D84075A82275D8
:10116B00B80275E690759B80759D0075D10E75BCA8
:10117B005875BB0675BA1175E88012059FD2AF1270
:10118B0008AC75360053DACF207E0343DA20307E6D
:10119B000343DA1043DA01C2D8C2711205B8D26127
:1011AB007B037A0CE55B70077A0CDB0302113112BF
:1011BB0005AE207003021131C270E55CC39402408E
:1011CB00E1E52F541F855E5DF55EB55DD5DAD5C2C1
:1011DB006153DACF207E0343DA20307E0343DA10EB
:1011EB00C2D8C27178A2E67008D274E52F54E0F52C
:1011FB002FC2757529001205B3307409C3E5299404
:10120B000A4002D2751205A478023074027800C32A
:10121B00E55C9840F0C2AF1205C81205C81205C8AC
:10122B00D2AF1205B8754C007888E6B4030261267C
:10123B001205A4788CE6C394015003021326E53003
:10124B00C394015003021326757CA5757DF12074A0
:10125B0035C3E55C94FF5003021326C2AF1205DDC4
:10126B00D2AF1205B3C3E55C940150EFC2AF1205C8
:10127B00C81205A91205C8D2AF1205B3C3E55C9419
:10128B00FF40E90217AE7F02D27F11311205B3C2C4
:10129B00AFC27F1131AE5CC3E55C947FD2AF50021D
:1012AB00613612059FC2AF1205DDD2AFDFDA1168CE
:1012BB00C3EE7897F61205B81217317F0AD27F1159
:1012CB00311205B3C2AFC27F1131AE5CC3E55C9482
:1012DB007FD2AF50E612059FC2AF1205C81205A907
:1012EB001205C8D2AFDFD61168EE24037896F6F854
:1012FB007997E7C394824003985006E82482789745
:10130B00F61205B81216441217601205B31131C349
:10131B00E55C94FF500241530217AE757C00757D5E
:10132B0000C3E55C954C4003855C4C1205B378011A
:10133B007988E7B403027805C3E55C984002413332
:10134B00C2AF1205DD1205DD1205DDD2AF1205B8F5
:10135B00753000E4F531F5320531E531F4703F05B8
:10136B0032789AE67819146012783214600D787D11
:10137B0014600878FA146003753200C3E5329840A4
:10138B001D120F2812059F1532753100789986733F
:10139B00C2AF1205DDD2AF789886731205B3120572
:1013AB00A9E52A7005307402213178012074027886
:1013BB0006C3E55C9840A17888E6C39403600312EA
:1013CB0005B3E52A7003021131C2AF120F28E4F501
:1013DB0022F523F524F525F526F567D2AF7885E6BA
:1013EB00C333F565E4F544F545F546F547F548F5A2
:1013FB0070F52CF52DF53775700875BB1012059F20
:10140B001208B030EDFDA8BDA9BEE97001F88871D6
:10141B001208B475700875BB10120FA9C2AF7561B5
:10142B00FF12094A852261852262852263D2AF753C
:10143B002201752401752501752601856069756A80
:10144B00017888E6B40307C27D307602D27DD2687C
:10145B00D269753300120E7D120EAE12096A120993
:0D146B007112096A12097112096A120BF15F
:101478001206BE120CE6120D2D120971120BE03085
:101488006E0312071A2066031208663066031208F4
:1014980096120CE6120D5C120971120BF1306E03F4
:1014A80012074F120CE6120DD5120971120BE0301B
:1014B8006E031207AD120CE6120E06120971120B1A
:1014C800F1306E0312080A120CE6120E7D12097131
:1014D8001208B0120BE0120CE6120EAE1208B4128B
:1014E8000971306932856461856462856069756AED
:1014F8000179187A0CC3E53399400FC269D26A8A18
:101508003585646185646302151FC3E55C940140F9
:10151800030214750215AD306A25206C22E53514D6
:101528007006C26AD26B8175F535C3E55C940140DB
:10153800030214757888E6C3940360030215AD7539
:10154800360078FA79A4E760027803C3E55F98501B
:1015580054307404E52A604D7888E6B40317207D7A
:1015680005207607A17D307602A17D206C07D26C1C
:1015780085646181B478F0306C058564617820C336
:10158800E5419850028175306C1BC26CC27D307683
:1015980002D27DD26A75351285646181750536E59A
:1015A8005C6002A1B0753600C2AF120F287887E6DA
:1015B800FE7602120FA97887EEF6E4F522F523F5F8
:1015C80024F525F526F565752C00752D00D2AF128A
:1015D80005B3120F2878A4E66006C292C291C290A1
:1015E800307409C3E536940440022131615E901AD3
:1015F8000D7820121686E520B4550CA3121686E540
:1016080020B4AA03021624757CA5757DF1120F3D3E
:10161800121644757C00757D00021643901A0378F3
:10162800807B0A121686A308DBF9901A0F788C7B48
:1016380019121686A308DBF9901A2822C2AF1216CF
:10164800C91216A6901A00740E12168BA3740912EA
:10165800168BA3741512168B901A0378807B0A12C6
:10166800168AA308DBF9901A0F788C7B1912168A50
:10167800A308DBF91216DC1216BA901A2822E49392
:10168800F622E6438F01538FFDFFC3E583941C4088
:101698000122EF857CB7857DB7F0538FFE22438FFB
:1016A80002438F01857CB7857DB7901A0DF0538F63
:1016B800FC22901A0D7455D18B901A0E74AAD18BF6
:1016C800227A3079D07820901A40D186E520F7091F
:1016D800A3DAF7227A3079D0901A40E7D18B09A3A0
:1016E800DAF922AB74A875BB01027980BB020279D2
:1016F80081BB03027982BB04027984BB0502798627
:10170800BB06027992BB07027987BB080279A3BBA3
:101718000902799CBB0A027988BB0B027989E8F730
:10172800227C051205B8DCFB22C2AF1205C81205DF
:10173800CF1205D61205DD1205A91205C81205CF6C
:101748001205D61205DD1205A91205C81205CF1219
:1017580005D61205DDD2AF22C2AF1205DD1205D6BD
:101768001205CF1205C81205A91205DD1205D612F9
:1017780005CF1205C81205A91205DD1205D61205F6
:10178800CF1205C8D2AF22AE74AF75C2AF1205C86A
:101798001205C81205C81205A9DEF21205DD1205E8
:1017A800A9DFF8D2AF22F131F129F1297574017559
:1017B8007501757600F18F7C05AD5C1205B8C3ED37
:1017C800955C70F5C3E55C9401400AC3E55C94FF41
:1017D80040320217EAD1EBD144F131C2AF75EF16AE
:1017E800F129DCD50576C3E5769403500280C6F16D
:1017F800290575E5741490009F93F808C3E575985A
:10180800500280AE1217291217290574C3E5749483
:101818000C5002809A120F3D121644C2AF75EF1693
:031828001217296B
:0319FD000210963F
:101A00000E0915090904FF03FF0A03010155AA0184
:101A1000FFFFFFFFFF03FFFFFF25D0285004FF0259
:091A2000007AFF0101000300FF40
:101A4000234F76736B794D52323041232020202072
:101A500023424C48454C4923463333302320202031
:101A60002020202020202020202020202020202076
:101C0000C2AFC2D353D9BF7581C043B20343FF8073
:101C1000752438752503B1DC7529A5752AF175E29F
:101C20004043F18053A47F75D4FFD2877DFA7803B7
:101C300079E67C10752200752300901DE97B0675FE
:101C400024987525013087028145208708D8FBD963
:101C5000F9DCF781B7308708D8FBD9F9DCF781B711
:101C6000B19CE493A3C39A6004DDC381B7DBDBB10D
:101C70008E6002812E7B08E493FAA3B16FDBF87AC1
:101C800030B16F752200752300B18EEAFCEBFDC305
:101C9000ED94FE400EB18E8A278B28ED30E0048A49
:101CA000828B83B18E7AC270D8C3ED94FE601950D6
:101CB000CEBD002BEC600F7520007521FF7529004B
:101CC000752A000200008100A827A9280809D80465
:101CD000D90281DCB192EA89AAF281CE0D81A3C337
:101CE000ED94035053EDA2E092007AC5C3E58294CF
:101CF00000E583941C508A200010438F02438F011B
:101D00008529B7852AB7F0300029A827A92808090E
:101D1000438F01538FFDD804D902A133C3E58394C7
:101D20001C4003A3A11689AAE28529B7852AB7F02A
:101D3000A3A116538FFC817F7AC1BD030CE493A34A
:101D4000FAB153DCF8B14B817F8181AA22AB23B178
:101D50006FEBFAEA6222752608C3E52313F523E543
:101D60002213F52250066323A0632201D526EAB18F
:101D7000DCB1DC75260AEAF4200102D287300102C8
:101D8000C287B1DCC3134002C201D526EB22B19257
:101D9000EAFB208702A192308702A197752608AE40
:101DA00024AF25C3EF13FFEE13FEB1E0B1DCC3EAAD
:101DB000133087024480FA30E703632201C3E5232E
:101DC00013F523E52213F52250066323A0632201B5
:101DD000D526D9E52265236523F52222AE24AF2539
:101DE0000E0FDEFEDFFCD20122424C48656C6934E6
:071DF000373164F3300601F6
:00000001FF
